:10000000F0C0E6CB09C108C107C106C105C104C1E2
:1000100003C102C101C100C1FFC0FEC0FDC0FCC0E0
:10002000CAC6FAC095CBF8C0F7C06AC4F5C0F4C020
:10003000F3C0F2C0ADC5B3C5CCC576C675C6DFC5C5
:1000400073C672C671C670C66FC66EC66DC66CC604
:100050006BC633C636C639C63CC63FC644C648C65C
:1000600057C64DC655C64BC64AC649C655C65CC6D8
:100070005BC6F1C5F4C5F7C5FAC5FDC502C606C61F
:100080000CC6DEC50EC611C612C615C650C64CC675
:100090004BC6C6C5C9C5CCC5EAC5EDC5F2C5F6C5D2
:1000A000CBC5CEC5D4C501C602C605C60600FF092C
:1000B00001A101150026FF0075088501950E0900B4
:1000C000B202018502951E0900B202018503953E28
:1000D0000900B202018504957E0900B2020185067D
:1000E000953E0900B20201C01201010100000008A2
:1000F000C016DF0500010102000109022200010112
:1001000000806409040000010300000009210101CE
:100110000001223C000705810308000A12011001BA
:1001200002000008C016E1050001010203010902F6
:100130004300020100806409040000010202010082
:1001400005240010010424020205240600010524F0
:100150000103010705830308006409040100020A82
:1001600000000007050102080000070581020800E1
:10017000000403090412036F006200640065007646
:10018000002E00610074003E0348006F00620062B0
:1001900000690065006C0065006B00740072006F00
:1001A000006E0069006B0061002E00680075003A67
:1001B0000020004100560052002D0044006F0070E6
:1001C0000065007200120361007600720064006F27
:1001D000007000650072000853544B3530305F32B8
:1001E000000011241FBECFEFD4E0DEBFCDBF11E071
:1001F000A0E0B1E0E6EBFAE102C005900D92AE326C
:10020000B107D9F714E0AEE2B1E001C01D92AC38FD
:10021000B107E1F759D04DCCF3CE20913801FC0164
:100220008381222379F0813019F428EE30E012C066
:10023000823021F02CE031E089E00DC02AEF30E07F
:1002400082E209C0813021F02EE231E083E403C074
:100250002CE131E082E13093A1032093A0030895C3
:10026000FC01808180768032C1F4809138019181D7
:10027000882369F0913011F0993021F582818093C3
:100280003601853011F483E019C081E017C0905227
:100290009230C0F41092370113C0803499F48181F8
:1002A000813049F492818091C00085FFFCCF90930A
:1002B000C60080E00895823029F484E080933701FD
:1002C0008FEF089580E008951F93CF93DF932EE082
:1002D00088E190E00FB6F894A895809360000FBE77
:1002E0002093600086E28093C40088E98093C10077
:1002F0003C9A449A3C98449886B182958F70809538
:1003000081708093380181E085B98FE384B988E0FA
:1003100088B984E387B983E18BB981E68AB9539AB6
:1003200020E048EB5BE004C0A895CA010197F1F713
:100330002150D1F7539883E085BD21E020936E00D2
:1003400082E88093800089E08093810081E090E0E2
:10035000909389008093880082E08093B00020937E
:10036000B1008093B30015D336D17894A89585D188
:1003700007D5809138018823C9F780910A0184FF4D
:10038000F5CFCEE2D1E010E004C089931F5F1830B2
:1003900049F0C5D397FFF9CF112321F480910001D3
:1003A000882321F3109300018EE291E0612F42D166
:1003B000DDCF1F93CF93DF93EC01162F899108D3E4
:1003C0001150E1F7DF91CF911F9108950F931F9383
:1003D000CF93DF93FC01162F90913701992359F4A5
:1003E0008BE480939203A1E0B1E087E001900D924D
:1003F0008150E1F727C0933009F530E0683009F00B
:1004000031E080913601853031F48181819580938E
:10041000360132961250909136019923A9F120812C
:100420008091C00085FFFCCF2093C6009F5F1150D4
:1004300019F4909336012CC03196EFCF892F81505B
:10044000823010F031E024C000E0683009F001E0B3
:10045000913011F0EF0109C0818180933601EF01E5
:100460002296125082E080933701809136018823D2
:1004700071F08881ADD28091360181508093360130
:10048000115029F02196F1CF1092360101C0302F82
:10049000832FDF91CF911F910F910895FF920F93BA
:1004A0001F93CF93DF938C01F62E90913701992300
:1004B00051F4D801E1E0F1E087E001900D92815024
:1004C000E1F727E081C09430E9F420E011C0E92F82
:1004D000F0E0EE53FC4F3281892F8F5F8093C2038F
:1004E000883C10F01092C203F80131938F012F5F06
:1004F0002F1508F069C09091C2038091C30398172B
:1005000031F762C09330B1F580913601853019F032
:10051000D801262F12C0F80181939091C3038091D6
:10052000C203292F281B981708F42853DF012D93A5
:100530002F2D225081E0809336018091360188234F
:1005400009F441C09091C2038091C303981789F1C7
:10055000E92FF0E0EE53FC4F3281892F8F5F8093BB
:10056000C203883C10F01092C2033C93215059F111
:100570001196E8CF892F8150823018F5913019F00B
:10058000E801162F0FC080913601E8018993BBD294
:1005900091118FEFF801818321961F2D125082E077
:1005A0008093370180913601882369F0B8D297FF94
:1005B00003C01092360107C08883115021F02196A4
:1005C000F5CF20E001C02F2D822FDF91CF911F9119
:1005D0000F91FF900895E9E6F0E0808183608083C9
:1005E000E89A83EC809392038093870308951F9386
:1005F000DC01162F80910B0184FF0AC080918703D4
:1006000098E8892780938703912FE8E8F3E007C0F3
:100610008AE580930B01F8CF8D91819391509923B6
:10062000D9F788E893E0612FCFD81C5F10930B01B6
:100630001F9108951F93DC01162F80910A0184FFFA
:100640000AC08091920398E8892780939203912FA2
:10065000E3E9F3E007C08AE580930A01F8CF8D91C2
:10066000819391509923D9F783E993E0612FACD816
:100670001C5F10930A011F9108950F931F93CF934E
:10068000DF936091A20316160CF0C6C080919F0301
:10069000CCE0D0E0C81BD109CA55DC4F6350809133
:1006A0009E03803118F4CE0184DEB4C08D3209F08F
:1006B00096C08AE580930901683009F0A3C088815B
:1006C000807609F07AC0109285038981882359F4D5
:1006D0001092860385E893E09093A1038093A00392
:1006E00020E892E075C0853021F48A818093A303CD
:1006F000FDC0863009F042C08B81813071F18230BB
:1007000061F1833041F58A81882349F481E791E0E2
:100710009093A1038093A00320EC94E059C0813012
:1007200019F485E791E010C0823049F487E891E040
:100730009093A1038093A00320EC9EE349C08330F3
:1007400009F0D6C085EC91E09093A1038093A003BB
:1007500020EC92E13DC0813229F4CE015EDD982F7C
:1007600020EC2FC0823209F0C3C08CEA90E0909355
:10077000A1038093A00320EC9CE32AC0883019F4E5
:1007800085EA93E00AC0893021F48A818093A50329
:10079000ADC08A3049F485E893E09093A10380933B
:1007A000A00320E891E014C08B3009F09FC083ECD7
:1007B000809392038093870399C0CE0151DD982FD7
:1007C00020E89F3F29F4888187FD9E812F771DC0F7
:1007D0008F818823D1F48E818917C0F016C0809153
:1007E000390187FD0FC0CE01F1DD8F3F21F48EE18D
:1007F0008093090104C0882311F020E004C020E0A8
:100800008FEF04C020E880E001C0892F20933901D8
:10081000809308011092A2038091090184FF5BC0BC
:10082000809108018F3F09F456C0182F893008F0D5
:1008300018E0811B809308018091390180FD02C07E
:100840000BE401C003EC8F5F8093390187FF26C062
:100850002091A0033091A10386FD05C0D901912FFD
:10086000EDE7F3E011C0ADE7B3E080E090E006C053
:10087000F901E80FF91FE491ED9301961817C1F7FC
:1008800005C08D91819391509923D9F7F901E10F1A
:10089000F11DF093A103E093A00309C0112339F0E7
:1008A0008DE793E0612FFADD182F893060F48DE732
:1008B00093E0612F89D7912F9C5F183041F08FEF23
:1008C0008093080104C08FEF809308019EE100939C
:1008D0007C03909309019AE089B18C7061F4915086
:1008E000D9F71092A30310929D0305C020E801C020
:1008F00020EC90E06DCFDF91CF911F910F91089583
:1009000078941F920F920FB60F9211242F933F935A
:100910008F939F93209178003091790080917C0093
:100920008F70E9F488E393E0821B930B25E0880F36
:10093000991F2A95E1F7865D9E4F181619061CF03F
:1009400081E090E006C021E08B39920714F08AE93B
:1009500091E0909389008093880081EC0AC0285F21
:100960003F4F84E0369527958A95E1F72093200143
:1009700080EC80937C0080917A00806480937A0080
:100980009F918F913F912F910F900FBE0F901F90CD
:10099000189580EC80937C00EAE7F0E08DE8808396
:1009A00080818064808308958091BC039091BD0311
:1009B000A091BE03B091BF030196A11DB11D80930C
:1009C000BC039093BD03A093BE03B093BF030895EF
:1009D000282F8091C103882321F410925402109291
:1009E00053028091530290915402009761F42B318D
:1009F00009F085C020933A0181E090E09093540281
:100A0000809353027CC031E08931930708F073C0B2
:100A1000FC01E65CFE4F2083FC013196F09354020A
:100A2000E0935302E430F105B1F480913D018093ED
:100A3000550280913C01809356028091550290911D
:100A40005602069690935602809355028A51914021
:100A500008F455C050C0E530F10521F42E3009F0FE
:100A60004AC04DC0E530F10508F449C080915502F7
:100A700090915602E817F90709F041C090E0AAE307
:100A8000B1E003C08D91982731973097D9F7109234
:100A9000540210925302992321F481E0809357026B
:100AA0002EC080EB80935D0280935E028BE1809389
:100AB000580280913B018093590210925A0282E0C1
:100AC00080935B028EE080935C021092720310921E
:100AD000710388E090E0909374038093730390E037
:100AE000E8E5F2E002C08191982732E0EF35F307A4
:100AF000D1F7908304C0109254021092530288ECF4
:100B00008093C10308952091730330917403809101
:100B1000710390917203281B390BC901089520912C
:100B20007303309174032115310519F4EFEFFFEFD2
:100B300019C08091710390917203FC01E85AFD4F36
:100B4000E08101969093720380937103821793075B
:100B500040F010927403109273031092720310927B
:100B60007103F0E0CF010895CF93DF93C2E0D0E0AE
:100B700080913F0180935D0210925E0290E0FC0143
:100B80003197EC33F10508F0CFC0E65EFF4F0994D2
:100B90008FE592E067ED71E085D7CBE0C8C0E091CA
:100BA000400120914101E63949F48091B100922F32
:100BB0009770887F982B9093B10004C0E73911F4A7
:100BC0002093B300F0E0EF71F070E45FFE4F2083FC
:100BD000AEC0E0914001E63921F4E091B100E77048
:100BE0000BC0E73919F4E091B30006C0F0E0EF71F3
:100BF000F070E45FFE4FE081E0935F0226C08091D9
:100C000040018093BF03809141018093BE03809196
:100C100042018093BD03809143018093BC0387C050
:100C200080E491E0F4D283C080E491E019D17FC0E8
:100C300080E491E0E5D279C080E491E0B1D175C063
:100C400080E491E02BD180935F02C3E070C080E428
:100C500091E09DD16AC080E491E00CD168C080E44D
:100C600091E00CD164C080E491E0C3D25EC080E426
:100C700091E060E009C080E491E06EE572E040E060
:100C80000AC080E491E061E0E8D14FC080E491E0E7
:100C90006EE572E041E096D144C080E491E061D11C
:100CA00044C080E491E054D140C009D1CCCF80E46D
:100CB00091E01DD1C8CF20D1C6CF80E491E0E5D32B
:100CC00034C080E491E0C8D332C080E491E079D4AC
:100CD0002CC080E491E060E009C080E491E06EE522
:100CE00072E040E00AC080E491E061E086D41DC07B
:100CF00080E491E06EE572E041E04AD312C080E406
:100D000091E02AD380935F0210926002C4E00FC08A
:100D100080E491E039D309C080E491E06EE572E0AF
:100D2000C0D2EC01219603C080EC80935E028BE17F
:100D30008093580280913B0180935902D0935A02CC
:100D4000C0935B028EE080935C021092720310925B
:100D500071032696D0937403C09373039E012150B0
:100D6000304090E0E8E5F2E004C0819198272150FE
:100D7000304021153105C9F79083DF91CF91089557
:100D800080915702882319F010925702EDDE0895E2
:100D9000982F969596958F5F891B8093C0038091BD
:100DA000C0038823E1F70895F89481E083BD86B5F8
:100DB000789486B5089578941F920F920FB60F928B
:100DC00011248F93F8948091C003882329F0809197
:100DD000C00381508093C0037894F89480912C01D3
:100DE000815080932C01882371F489E480932C0135
:100DF00078948091C103882339F08091C103815098
:100E00008093C10301C078948F910F900FBE0F9013
:100E10001F901895982F9F5F86958695981B9093A5
:100E2000C0030895382F9BB19F799BB92B9A2B98BB
:100E300080E028E0880F4F99816067FD906437FD5E
:100E400090629BB92B9A9F792B98215019F0330F00
:100E5000660FF0CF9BB92B9A2B982B9A2B9808955D
:100E60002A98229A459A8BB18F798BB9289A4598FE
:100E70002D98089581E080937503089508951F9338
:100E8000182F8CE464E0CEDF812F886660E0CADF33
:100E9000812F8C6660E0C6DF1F910895FC01E08120
:100EA000EE2311F480E009C0E13011F482E105C0C5
:100EB000E23011F080EC089582E0E1DF089580E1F6
:100EC000DEDF08950F931F93182F062F8CE468E040
:100ED000A9DF8CE0612FA6DF802F886660E0A2DFAB
:100EE000802F8C6660E09EDF1F910F910895FC01BA
:100EF000808160E0E7DF089580E060E1E3DF08954E
:100F00008091760387DF06C08091C003882311F4A7
:100F100080E808954F9BF8CF80E008950F931F93CA
:100F2000082F142F8CE47EDF8CE2602F7BDF812F73
:100F3000846660E077DF812F8C6660E073DFE0DF3E
:100F4000182F8CE460E06EDF812F1F910F910895C0
:100F5000FC01838180937603818160E240E0DEDFE3
:100F60000895FC018381809376038081882311F4A6
:100F700040E009C0813011F440E105C0823011F039
:100F800042E101C042E0818160E4C8DF0895FC01D4
:100F9000828180937603818160E240E0BFDF089523
:100FA000FC018281809376038081882311F440E0E4
:100FB00005C0813011F042E001C040E1818160E470
:100FC000ADDF0895DF92EF92FF920F931F93CF93BF
:100FD000DF93FC01DB01D42E908181811C928C0176
:100FE000442311F462E001C063E07D010894E11C38
:100FF000F11C8CE417DFE80120C02197A8958CE054
:101000006091BC030FDF8CE16091BD030BDF88E6CC
:1010100060E008DF8CE660E005DFF70181937F0187
:10102000DD2051F488E760E0FDDE8CE760E0FADE69
:10103000F70181937F012197B7DC2097F1F6F70143
:10104000108298012E5F3F4FC901DF91CF911F9110
:101050000F91FF90EF90DF9008956F927F928F92A3
:101060009F92BF92CF92DF92EF92FF920F931F93C6
:10107000CF93DF93FC01C62E838180937603E180BA
:10108000B2808B2D869581958770DD24DA9402C01D
:10109000D69481508823E1F7CC2011F061E102C0A1
:1010A000D69460E18F010C5F1F4F8CE4BBDEFF2400
:1010B0006B2C772481E0882E912C86209720A89590
:1010C0008CE06091BC03AEDEE801219681149104AE
:1010D00059F1F80160818E018CE2A4DECC2029F068
:1010E0008DE660E09FDE8CE609C0FE0161918F0114
:1010F0008CE398DE8DE760E095DE8CE760E092DEC1
:101100008091BC038F5F8D21D9F5B7FE39C08CE18A
:101110006091BD0387DE84E660E084DE8CE660E0FB
:1011200081DEEEDEF82E2CC08CE16091BD037ADE0C
:10113000F80160818E018CE275DECC2041F08DE6F5
:1011400060E070DE84E660E06DDE8CE613C084E66D
:1011500060E068DE8CE660E065DED2DEF82E882393
:10116000D9F4FE0161918F018CE35CDE84E760E0DD
:1011700059DE8CE760E056DEC3DEF82E882361F48A
:1011800013DCCC2011F4EA9419F0EA9409F097CF1B
:10119000892811F066FE03C08CE460E043DE8F2DE9
:1011A000DF91CF911F910F91FF90EF90DF90CF9043
:1011B000BF909F908F907F906F9008951F93182FEE
:1011C0008CE460E82FDE84E660E02CDE8CE660E0F4
:1011D00029DE80917603882319F092DE182F03C050
:1011E000812FD6DD10E08CE460E01CDE812F1F91A2
:1011F0000895FC018181809376038AE0DFDF089502
:10120000FC018081809376038181D8DF089510925C
:1012100075032D9AE0EBF0E080818F7B8083459A07
:101220002898579A87E0C0DD459822982A9A82E04C
:10123000BBDD579888E3B8DD0895DF92EF92FF9207
:101240000F931F93CF93DF93EC01E62ED09077039B
:10125000F89408B10F7E10E018C0188188E0F82ECD
:1012600017FD006108B978948D2D9EDDF894429A9F
:10127000110F0F7E339B116078948D2D95DDF894BE
:101280004298FA9469F72196EA94EE2031F778941F
:10129000812FDF91CF911F910F91FF90EF90DF9001
:1012A0000895AF92BF92CF92DF92EF92FF920F9389
:1012B0001F93CF93DF93EC015B0188811A81811723
:1012C00008F4182FCE010396612FB7DF750108943B
:1012D000E11CF11C00E0C12EDD2412C02C0D3D1DCF
:1012E0002D5F3F4FCE01820F931F61E0A6DF982F45
:1012F0008981081718F4F70191937F01A8950F5F72
:10130000202F30E0888190E08C199D09281739073B
:101310002CF30BC01092780388E793E061E08DDF37
:10132000F70181937F01A8950F5F8981081790F3DA
:10133000F5011082F7011082298130E02E5F3F4FC6
:10134000C901DF91CF911F910F91FF90EF90DF9036
:10135000CF90BF90AF9008951F93CF93DF93EC0190
:10136000019668816ADF182F2881243040F4822F8B
:1013700090E0019664E0621B8C0F9D1F5EDF812F61
:10138000DF91CF911F91089564E057DF80E00895C9
:10139000AF92BF92CF92DF92EF92FF920F931F9383
:1013A000CF93DF93EC017B01C42E10927B03442387
:1013B00089F48091BF0387FF0DC08DE4809378038B
:1013C000109279038091BE0380937A0388E793E0BB
:1013D00064E033DF9881898157010894A11CB11C16
:1013E000F7011082DA80EC0100E010E01FC0A89540
:1013F0008091BD03809379038091BC0380937A032D
:10140000CC2041F400FF03C0F8E0DF2A03C087EFDF
:10141000D82201C0C9DAD092780388E793E064E06B
:101420000CDFF50181935F010F5F1F4F0C171D0744
:10143000F0F2EC0EFD1EF70111829E012E5F3F4F70
:10144000C901DF91CF911F910F91FF90EF90DF9035
:10145000CF90BF90AF9008950F931F938C0188B1E8
:101460008B7E88B9459AF801808192DCE0EBF0E050
:1014700080818F7B80832C98249A45982D98F80141
:10148000818186DC1F910F910895DF92EF92FF9288
:101490000F931F93CF93DF93EC0180912401498137
:1014A0004C9902C08DE01CC0882311F0813019F4E2
:1014B0001092770317C0823011F481E011C083309D
:1014C00011F482E00DC090E001969C0135952795BE
:1014D0003595279534E0959587953A95E1F7820FF4
:1014E000809377032D9A88B18B7E88B9459A24988A
:1014F0002C9A8091B00080648093B000842F48DCE7
:101500008091770351DC4598809177034DDC459AB3
:101510008A813EDC27E0E22EF12CEC0EFD1E10E26B
:1015200094E0D92E1DC0A895C7016E8186DE082FD4
:101530002E81243040F4822F90E007966D2D621B9F
:101540008C0F9D1F7ADE8D81081711F480E01AC080
:10155000429A8091770328DC42988091770324DCBB
:10156000115008F788B18B7E88B9459A80E010DC6D
:101570008091B0008F7B8093B0002C98249A45987E
:101580002D9880ECDF91CF911F910F91FF90EF90FC
:10159000DF9008951F933EDC10EF06C08091C003DA
:1015A000882311F481E80BC010937803109279031B
:1015B00088E793E064E041DE80FDF0CF80E01F919A
:1015C0000895FF920F931F938C01FC01F080029607
:1015D00064E033DEF8018181882341F0F9E0FF15F2
:1015E00010F06AE0F62E8F2DD5DF03C08F2DD0DBF3
:1015F00080E01F910F91FF9008956F927F928F92DC
:101600009F92AF92BF92CF92DF92EF92FF920F9391
:101610001F93CF93DF93EC01662EF88019818A81A6
:1016200080FD04C0E4E07E2E08E003C070E2772E67
:1016300000E4662099F48091BF0387FF0FC08DE41A
:1016400080937803109279038091BE0380937A038C
:1016500010927B0388E793E064E0EFDDC12EDF2C7E
:1016600046010894810891085E01EE24FF245CC0C5
:10167000A8958091BD03809379038091BC038093EA
:101680007A03F501818580937B031C81662021F418
:10169000177FE0FE02C0186087D91093780388E7AF
:1016A00093E064E0CADD8A8180FF0CC0E814F9048D
:1016B00090F187FF30C08D818093780388E793E0B5
:1016C00064E0BBDD9A81872D8923F1F0F501118556
:1016D0008F811817F1F088851817D9F08E81877FD0
:1016E000E0FC8860809378038B8194DB06C0809156
:1016F000C003882311F480E80FC088E793E064E01A
:101700009CDD8117A1F707C0902319F08B8142DF80
:1017100003C08B813DDB80E00894A11CB11C8823B1
:1017200041F40894E11CF11CEC14FD0408F4A0CF72
:1017300080E0DF91CF911F910F91FF90EF90DF90AC
:10174000CF90BF90AF909F908F907F906F900895B3
:101750001F920F920FB60F9211242F938F939F9386
:10176000EF93FF932091C600E091C3039E2F9F5FEC
:10177000983C08F090E08091C203981731F0F0E0B7
:10178000EE53FC4F22839093C303FF91EF919F91FF
:101790008F912F910F900FBE0F901F901895A82F2B
:1017A000B92F80E090E041E050EA60956F5F58F417
:1017B0002D9138EF82279795879510F084279527EC
:1017C0003F5FC8F3F3CF0895EADF8D939D930895AB
:1017D000CF93CFB7CF934B9BFECF4B9B09C04B9B77
:1017E00007C04B9B05C04B9B03C04B9B01C0A6C0D1
:1017F000DF93C0919F03DD27CA55DC4F4B9B02C08E
:10180000DF91EBCF2F930F931F9309B12FEF03FBC2
:1018100020F94F933F9319B14FEF012703FB21F9B3
:101820003BE031C04E7F012F19B1216028C0102F3D
:101830004D7F2260000009B129C04B7F2460012F39
:10184000000019B12BC019B1477F28602AC04F7E14
:1018500009B120612CC04F7D19B120622FC04F7B90
:1018600009B1206432C0422709B149934FEF00000B
:10187000102713FB20F919B11C70C9F1297F91F2CF
:10188000012703FB21F909B1237F89F2315058F177
:10189000102713FB22F919B1277E79F2012703FBE8
:1018A00023F92F7C81F209B1102713FB24F92F793A
:1018B00071F200C019B1012703FB25F92F7359F20A
:1018C00000C009B1102713FB26F9223040F200C0F6
:1018D00019B1012703FB27F9243028F64F77206838
:1018E00019B10000F9CF11E01CBB00271CC03B5010
:1018F0003195C31BD04011E01CBB0881033C11F1A2
:101900000B3401F120919D031981110F1213EDCFBA
:101910004A81441F093659F10D3211F0013E29F771
:101920004F7009F0042F0093A4033F914F911F9132
:101930000F912F91DF91CCB3C0FD4DCFCF91CFBF91
:10194000CF9118950091A403002379F31091A2037D
:101950001123F9F53430FAF13093A20300939E037A
:1019600010919F033BE0311B30939F0334C00091E3
:10197000A203013074F50AE54F7049F43091090172
:1019800034FD2BC000930901CCE7D3E02AC04330DB
:1019900049F030910A0134FD20C000930A01C2E9E8
:1019A000D3E01FC030910B0134FD17C000930B0131
:1019B000C7E8D3E016C0052710E00BB91FC0052704
:1019C00022C0052727C005272CC0052710E00BB92A
:1019D00033C04AE503C042ED01C0432FC4E1D0E06B
:1019E00032E01AB11C605B9A0BB11AB95F935CE0EC
:1019F00020E820FF05270BB9279517951C3FD8F63F
:101A000020FF052727950BB917951C3FC0F620FF2F
:101A10000527279517950BB91C3F98F620FF05273A
:101A2000279517951C3F0BB970F600C0499120FF10
:101A300005270BB9279517951C3F38F620FF05277A
:101A400027950BB917951C3F38F520FF05272795DB
:101A500017950BB91C3F10F520FF05272795179503
:101A60001C3F0BB9E8F4242F3A9519F6037F5F91D8
:101A70000BB91091A303110FC651D04011F0109370
:101A80009D0311E01CBB08601AB1137F402F437FF8
:101A90000BB91AB94BB949CF0527D3CF0527D8CFF2
:101AA0000527DDCFFB01DC0105900D920020E1F759
:061AB0000895F894FFCF39
:101AB6000180250000000008FF5A5A5A0000000065
:101AC60000000000000000000000000001020A0003
:0E1AD600320001800200AA00000000000100A2
:00000001FF
